:100000002BC045C044C043C042C041C040C03FC0F7
:100010003EC03DC0CBC23BC03AC039C038C092C21E
:10002000A9C292C2A7C292C2A5C2A4C2A3C290C2D0
:10003000A1C290C29FC290C29DC29CC29BC28EC2EE
:1000400099C28EC297C28EC295C294C293C28CC20C
:1000500091C28CC28FC28CC211241FBECFE5D1E0E9
:10006000DEBFCDBF10E0A0E6B0E0E2EDF6E002C0FA
:1000700005900D92A236B107D9F710E0A2E6B0E0E4
:1000800001C01D92A736B107E1F7CBD220C3B8CF8C
:1000900087B3876087BB08958FB980E48EB98BE101
:1000A0008DB9769BFDCF0895C0988FB980E48EB945
:1000B0008BE18DB9769BFDCF6FB980E48EB98BE172
:1000C0008DB9769BFDCF88B391E0892788BB0895D1
:1000D0001F93182F81E0612FE7DF82E0612FE4DFBB
:1000E00083E0612FE1DF84E0612FDEDF85E0612FB7
:1000F000DBDF86E0612FD8DF87E0612FD5DF88E086
:10010000612FD2DF1F9108958AE06FE0CDDF8BE091
:1001100067E0CADF89E060E0C7DF80E0D9DF8CE01C
:1001200061E0C2DF08951F93182F83E0612FBCDFC9
:1001300084E0612FB9DF85E0612FB6DF86E0612FB3
:10014000B3DF87E0612FB0DF88E0612FADDF1F9163
:1001500008951F93182F81E0612FA6DF82E0612FA1
:10016000A3DF1F91089581E06FEF9EDF82E06FEFC4
:100170009BDF83E06FEF98DF84E06FEF95DF85E032
:100180006FEF92DF86E06FEF8FDF87E06FEF8CDF3E
:1001900088E06FEF89DF089581E06FEF85DF82E00F
:1001A0006FEF82DF089581E060E07EDF82E060E053
:1001B0007BDF08951F9380E0B6DF8FEFCADF1091D9
:1001C00061008AE0612F70DF88EE93E028EC30E078
:1001D000F9013197F1F70197D9F7809166008823EB
:1001E00011F4115001C01F5F1093610080916100F4
:1001F000813019F48093660004C08F3011F410929E
:1002000066001F910895AF92BF92CF92DF92EF9256
:10021000FF920F931F93CF93DF938AE06FE044DF49
:1002200080E056DF11E021E0A22EB12C90E3C92E30
:1002300095E7D92E88ECE82EF12C1FC0C5010C2EB5
:1002400002C0880F991F0A94E2F7080F812F602FD0
:100250002BDF133040F482EC91E0F7013197F1F796
:100260000197D9F703C0C6010197F1F72196C8306D
:10027000D10521F71F5F193021F000E0C0E0D0E088
:10028000DDCF84EC99E028EC30E0F9013197F1F70B
:100290000197D9F7DF91CF911F910F91FF90EF90C8
:1002A000DF90CF90BF90AF900895CF92DF92EF9202
:1002B000FF920F931F93CF93DF938AE06FE0F4DEFA
:1002C0008FEF06DF08E041E0C42ED12C30E3E32EAF
:1002D00035E7F32E16C0C6010C2E02C0880F991FF9
:1002E0000A94E2F7181B802F612FDEDEC701019709
:1002F000F1F721978FEFCF3FD80769F70150023010
:1003000021F01FEFC7E0D0E0E6CF84EC99E028ECC5
:1003100030E0F9013197F1F70197D9F7DF91CF91EB
:100320001F910F91FF90EF90DF90CF900895CF92A3
:10033000DF92EF92FF921F93CF93DF938AE06FE0FB
:10034000B3DE80E0C5DE10E0C0E0D0E0E1E0CE2E1C
:10035000D12C78ECE72EF12CC6010C2E02C0880FB0
:10036000991F0A94E2F7180F81E0612F9DDE84EC5B
:1003700099E0F7013197F1F70197D9F72196C83045
:10038000D10551F710E0C0E0D0E061E0C62ED12CDD
:1003900058ECE52EF12CC6010C2E02C0880F991FD7
:1003A0000A94E2F7180F82E0612F7EDE84EC99E078
:1003B000F7013197F1F70197D9F72196C830D105A8
:1003C00051F7DF91CF911F91FF90EF90DF90CF9089
:1003D0000895CF92DF92EF92FF921F93CF93DF9316
:1003E0008AE06FE061DE8FEF73DE1FEFC0E0D0E0E8
:1003F00081E0C82ED12CB8ECEB2EF12CC6010C2ECE
:1004000002C0880F991F0A94E2F7181B81E0612F40
:100410004BDE84EC99E0F7013197F1F70197D9F7BA
:100420002196C830D10551F71FEFC0E0D0E0A1E020
:10043000CA2ED12CF8ECEF2EF12CC6010C2E02C0E6
:10044000880F991F0A94E2F7181B82E0612F2CDEB7
:1004500084EC99E0F7013197F1F70197D9F72196EC
:10046000C830D10551F7DF91CF911F91FF90EF90E8
:10047000DF90CF900895CF92DF92EF92FF921F937B
:10048000CF93DF9380E024DE11E021E0C22ED12C57
:1004900098ECE92EF12C17C0B6010C2E02C0660FA5
:1004A000771F0A94E2F7812FFFDD84EF91E0F701D7
:1004B0003197F1F70197D9F72196C830D10561F747
:1004C0001F5F193019F0C0E0D0E0E6CFDF91CF9187
:1004D0001F91FF90EF90DF90CF9008951F931091A0
:1004E0006500133061F0143018F4113071F405C058
:1004F000153039F0173049F406C083E307C086E6AB
:1005000005C08CEC03C089E901C08FEF0CDE80E6EA
:100510009AEE0197F1F7812F8F5F80936500883005
:1005200010F0109265001F9108951F9310916400C0
:10053000812F90E0FC013197ED31F105D8F4E15FB6
:10054000FF4F099488E817C08CEC15C08EEE13C0DD
:1005500084E411C086E60FC087E70DC082E20BC0BD
:1005600083E309C08BEB07C081E105C089E903C0C3
:100570008DED01C08FEFD7DD80E29EE40197F1F7AA
:10058000812F8F5F809364008F3110F01092640090
:100590001F91089588B3886188BB0895789480E19D
:1005A00089BF8CE083BF8EEF89BD08951F920F92A3
:1005B0000FB60F9211248F9380916200882359F512
:1005C00080916300882339F580916000813021F0AB
:1005D00080916000823039F4B49B05C081E0809343
:1005E00062001092600080916000882321F0809169
:1005F0006000823039F4B49905C081E080936200D4
:100600008093600080916200882329F4B39903C02D
:1006100081E0809363008F910F900FBE0F901F9029
:100620001895FF920F931F93CF93DF9388B3886140
:1006300088BB87B3876087BB67DD789480E189BF1B
:100640008CE083BF8EEF89BD88E893E128EC30E031
:10065000F9013197F1F70197D9F700E0C8ECD0E044
:100660001091600080916200F0906300813069F425
:10067000113051F5F8945BDE10926200789405C059
:10068000F894C1DD10926200789481E0F816A1F42C
:10069000F8941092630088EE93E0FE013197F1F731
:1006A0000197D9F7112339F4002319F4FEDD01E095
:1006B00002C0A9DD00E07894113021F0002311F48C
:1006C0000DDFCECF77DDCCCF1123F9F6D9CFF8945B
:0206D000FFCF5A
:0206D200020F15
:00000001FF
